:060000000C9448000C9472
:1000060000000C9400000C9400000C9400000C946A
:1000160000000C9400000C9400000C9400000C945A
:1000260000000C9400000C9400000C9400000C944A
:1000360000000C9400000C9400000C9400000C943A
:1000460000000C9400000C9400000C9400000000CA
:10005600003FCDCC4C3D0AD7A33B6F12033A17B7EE
:100066005138ACC5A736BD37063580C0000054658B
:100076006D703D25352E316620430000020060017B
:1000860070000200640172000000F894EE27ECBBD9
:10009600F1E0FBBFEBBFE5BFF8E1F1BDE1BD8DE0EF
:1000A600A2E0BB27ED938A95E9F780E094E0A0E60D
:1000B600ED930197E9F7E2E8F0E0859195910097D5
:1000C60061F0A591B59105901590BF01F0010590DD
:1000D6000D920197E1F7FB01F0CFEFE5EDBFE4E00C
:1000E600EEBFC0E6D1E00C948300E881E06CE7B98E
:1000F600369A349BFECF349AE4B1F5B12196089531
:100106002E97E0E0EBBBE1E0E7BBE0ECE7B9E6E821
:10011600E6B9E0E1EA930E945405E0E0EA930E9422
:1001260078008F01D801E4E0F0E00E9428070E94E1
:10013600A005E883F9836A837B83A881B9818A81D4
:100146009B81E0E0F0E068EC71E40E94250909F08B
:1001560010F40C94B000C09A01C0C098FE01349609
:10016600FA93EA93E4E7F0E0FA93EA930E94A5058E
:100176000E948C0784E00E947A0428960E94030558
:10018600E0E0EA93EA930E94EF04FE013496FA93C4
:10019600EA930E943305E8EEF3E0FA93EA930E94AD
:1001A6009E06BBCFFFCF5F9BFECFECB108955D9B54
:1001B600FECFE881ECB9219608951A930A93AC8193
:1001C600BD810E947C073097B9F0AA81BB810E944D
:1001D6007C078F01309749F00230E0E01E0758F0A7
:1001E600F80131978F01ED93FC93AC81BD810E949C
:1001F600AA05AE81A08304C0EE81EA930E94DA00CC
:10020600198108812796089524971A930A93A88539
:10021600A73010F0E6E0E887E885F0E0A4E5B0E076
:100226000E94F206EA0FFB1F0E9486070E94B10594
:100236000E9444080E94B60510E0E0E0F0E060E8A5
:100246007FE30E94BB050E94C0050E94250940F07D
:100256000E94C5050E9492080E94BB051F5FF3CF4E
:10026600103029F40E94CE05E0E3EC9322C0E12F82
:100276001150E030F1F00E94C5050E94D5050E949C
:10028600BB050E94C0050E94E0080E94D3070E2FFE
:100296000E94CE050E94E105AA81BB818C819D81C9
:1002A6000E94A0050E9492080E94B1050E94E705DF
:1002B600DECFE885E03029F4AE81BF81E0E0EC9343
:1002C60025C00E94CE05EEE2EC93E885E150E88772
:1002D600EF5FC1F00E94B1050E94EC050E94B605D1
:1002E600E985FA856B857C850E94D1070E2F0E94D1
:1002F600CE050E94E1050E94B1050E94A0050E945C
:10030600E705E3CFAE81BF81E0E0EC931981088178
:100316002D96089524970E944F09E0E0F0E060E8EA
:100326007FE30E94F305AB85A73010F0E6E0EB878C
:100336001B85E12F1150E03029F00E94F8050E943C
:10034600F305F7CF0E94FD050E94450931F430E020
:100356000E94F8050E94F30534C03B850E94020600
:1003660009F010F40C94C4010E94F8050E94F305EC
:100376000E94020628F00E940A060E940F06F8CF85
:100386000FC00E94020640F40E940A060E94EC0575
:100396000E941B063150F5CF0E94F8050E94F30516
:1003A6000E94FD05A0E0B0E080E09FE30E944408C3
:1003B6000E941B060E94020620F00E940A060E9466
:1003C6000F0610E0EB85E117B8F1AC81BD818E8197
:1003D6009F81E0E0F0E060E271E40E94D5050E94B2
:1003E600F3050E94A5050E940A060E94E0080E94E5
:1003F600D3070E2F0E942006E02FE05DEC93E02F3E
:10040600FF27662777270E940A08AC81BD818E8167
:100416009F810E9492080E940A060E9491070E94EC
:100426003D080E941B06E12F1F5FE03059F60E942F
:100436002006EEE2EC93C6CF0E942706AA85A0838B
:1004460030302CF40E942006EDE2EC9331953A30E0
:100456004CF00E942706BF01A32FEAE00E94100776
:100466000E942E060E942706BF01A32FEAE00E94E3
:1004760052070E942E06A885B985E0E0EC930E94FB
:10048600560960960895EF972F970E944D0910E040
:10049600FE01EC5AFF4F0190F081E02DE88BF98BBD
:1004A600DE01A65ABF4F0E94AA05E4912E2FE03026
:1004B60011F40C947504E12FF0E0309739F42532ED
:1004C60011F411E002C00E9435060BC2E130A0E033
:1004D600FA07C1F4253219F40E94350601C212E06A
:1004E600E0E0EB8B00E02D3211F401E0FAC12B3293
:1004F60019F4EBE2EB8BF5C1203219F4E0E2EB8B59
:10050600F0C104C0E230A0E0FA0739F450E013E08D
:10051600203311F40068E5C104C0E330A0E0FA0717
:10052600A9F4203310F02A3308F00AC0A52FEAE018
:10053600EA9FF0015E2FE22FE053F0E05E0FD1C19B
:1005460040E02E3211F414E0CCC114C0E430A0E037
:10055600FA07B1F4203310F02A3308F00BC000621A
:10056600A42FEAE0EA9FF0014E2FE22FE053F0E0DD
:100576004E0FB7C12C3619F4026015E0B2C106C0A1
:10058600E530A0E0FA0711F00C947404E22FF0E0D5
:10059600E336A0E0FA0731F40E944406E4810E94A3
:1005A6004D069EC1E534A0E0FA0721F0E536A0E04D
:1005B600FA0709F406C0E636A0E0FA0711F00C9433
:1005C6002C03FE017496EA87FB870E944406349644
:1005D600DF010E9480070E945C06DF01CB010E94BA
:1005E600490924F0AB89AB3249F012C00E9461067A
:1005F6000E949E070E945C06EDE2EB8B07FF04C09B
:10060600EB890E944D0604C00E946606AB89A08352
:1006160005FF46E0263661F40E9461060E948C07BB
:100626004A93EF85F889FA93EA930E9407010CC072
:100636000E9461060E948C074A932A93E889F989E9
:10064600FA93EA930E948D01FE0174960E946D064C
:1006560022C0E337A0E0FA0739F40E9444060E945C
:1006660075060E946D0610C0E037A0E0FA07C1F4D7
:100676000E9444060E947506EA87FB87FA93EA936E
:100686000E9495051E2F08600F77403011F0411724
:1006960008F001C0142F40E0E0E0EA8B30E079C0BA
:1006A600E436A0E0FA0721F0E936A0E0FA0711F4F3
:1006B600046004C0E537A0E0FA07A1F4EAE0EA8B9B
:1006C60001FF08C0E0E0FAEC6AE97BE30E941B0642
:1006D6001AE027C0E0E1F7E260E070E00E941B0646
:1006E60015E01FC0E835A0E0FA0711F4086006C05F
:1006F600E837A0E0FA0711F00C947304E0E1EA8B06
:1007060001FF08C0E0E0F0E060E070E10E941B0637
:1007160018E007C0E0E0F0E160E070E00E941B0630
:1007260014E0403011F00F7701C041E001FF07C02F
:100736000E9444063496DF010E9480070FC002FF24
:1007460007C00E9444060E9475060E94FD0606C068
:100756000E9444060E94750666277727EE83FF836C
:100766006887798702FF14C00E947A060E944909A9
:1007760044F40E9461060E94EA060E945C06EDE2CD
:10078600EB8BEB89E03019F01F5F4F5F01C00B7FE9
:10079600342F00FD14C0151710F4351708F00FC0DC
:1007A60007FF08C002FF04C00B7F2B89115001C050
:1007B60020E301C020E20E9435065150ECCF141709
:1007C60088F4006102FF06C00E947F0609F05150BE
:1007D60011504150E0E30E944D06503009F051504F
:1007E6004150EDCF312FEA89E03011F53030F9F084
:1007F60003FF04C00E946606E49105C0AA85BB8576
:10080600ED91AA87BB87EA93FE01E95AFF4F019053
:10081600F081E02DFA93EA93FE017396FA93EA9338
:100826000E94E000503009F051503150DFCF4FC0E8
:100836000E94FD050E947A060E942D072E2F2A305F
:1008460030F003FF02C0295C01C0295A01C0205DB7
:1008560004FD1FC0213350F40E940A06A130E0E0D7
:10086600BE07E0E08E07E0E09E0709F40BC04317E1
:1008760040F4531710F000FF01C010C020E207FF3C
:1008860008C020E3006102FF04C00E947F0609F051
:1008960051500E943506503009F0515031500E9497
:1008A600FD050E947A060E945E070E945C06EA89A0
:1008B600F0E00E940A060E94FD060E942D070E9493
:1008C6001B060E94FD050E94450909F0B1CF00FFF5
:1008D60007C0503029F05150E0E20E944D06F9CF92
:1008E60010E0DECD0E945409EF966D960895FF92B2
:1008F600F82E22971A930A93DE010E94E2068D01D2
:10090600DE0116960E94E2060E947C07EA83FB83BC
:10091600DE0114960E94E2060E947C07FA93EA938F
:100926001A930A93FE013696FA93EA93E0E0F0E012
:10093600FA93EA930E944602AA81BB81E0E0EC9317
:10094600198108812496FF900895FFE0FA95F1F742
:100956000895A1B3AF70A1BB919A90980E94A80484
:10096600929A0E94A804A0B392980E94A804929A10
:100976000E94A8049298A7FDF1CF0895A07FAB2B03
:10098600A2BB929A0E94A80492980E94A804089575
:100996009198A1B3A76FA1BBB2B3BF70A8810E9403
:1009A600C104A881A2950E94C104919A2196089536
:1009B600929A0E94A804E0B392980E94A804E07F4D
:1009C60008950E94A8040E94DB04AE2F0E94DB0457
:1009D6009198E295EA2B08950E94AC04E881F0E034
:1009E600E05AFE4FE081AE2FE981F0E0B0E0EA0F79
:1009F600FB1FEA930E94CB045980488022960895F3
:100A06000E94AC04E2E0EA930E94CB040E94AC048C
:100A1600ECE0EA930E94CB040E94AC04E1E0EA9386
:100A26000E94CB04E0E04E2E5E2E0895EF93FF93D6
:100A3600A8816894AA3021F0E8945394751438F488
:100A46004394E0E0EA934A920E94EF042EF081DF9D
:100A5600909AA881AA939CDFFF91EF912196089521
:100A66001A93A981BA81ED91A983BA831E2FE0302A
:100A760021F01A930E941905F4CF18812396089540
:100A8600AA27BB271197F1F708959198A1B3A76FED
:100A9600A1BBB2B3BF70A8810E94C104919A2196EE
:100AA6000895929890987880E881E058E0936201E2
:100AB600E881E054E09363010E9493060E94930646
:100AC6000E9493060E944305E0E2EA930E944805CD
:100AD6000E944305E8E20E949906E4E00E94990616
:100AE600E5E80E949906A1B3AF70A1BB919A0E9456
:100AF600E404E53011F0E0E009C00E94AC04E6E051
:100B0600EA930E94CB040E940305E1E02196089532
:100B1600A991B991EE27FF276D91662311F03196C1
:100B2600FBCF0895AA27BB27E991F99105900020EC
:100B360011F01196FBCFFD0108950E94FD060E945B
:100B46000A080895EC81FD816E817F810895ED91FB
:100B5600FD913196FE93EE9331970895A985BA8556
:100B66008B859C850895E987FA876B877C8708952E
:100B7600EA83FB836C837D830895EA81FB816C8124
:100B86007D81ECCFAA81BB818C819D81E0E0F0E084
:100B960060E271E40895AE81BF811196AE83BF8392
:100BA600119708950E94E008A0E0B0E080E09FE37E
:100BB6000E9444080E948C070C94D906E02FE05D41
:100BC600EC93E02FF0E008950E9491070E943D0803
:100BD600CACFE0E0F0E060E271E40E949208089576
:100BE600EC83FD836E837F830895AC81BD818E8106
:100BF6009F81EFCFEC85FD856E857F850895A2DF09
:100C0600AC85BD858E859F850E9425090895AC8596
:100C1600BD858E859F850895E0E0F0E060E271E491
:100C26000E94E008EC87FD876E877F873F5F089507
:100C3600EC87FD876E877F870895A885B98511960D
:100C4600A887B98711970895E885F9853196E887C9
:100C5600F98731970895F0E0E7FDFFEFF096DB01A5
:100C6600EC9308952A93FE01E95AFF4F0190F08113
:100C7600E02DFA93EA93FE017396FA93EA930C94A5
:100C8600E000DE01A85ABF4FED91FD913497FE9327
:100C9600EE930895EA93FE01E95AFF4F0190F08121
:100CA600E02DFA93EA93FE017396FA93EA930C9475
:100CB600E000EE83FF83688779870895EE81FF81E0
:100CC600688579850895EA85FB853196EA87FB87ED
:100CD60031970895EA87FB87FA93EA930E948B057A
:100CE6001E2F08953496DF010E947C070895AE8179
:100CF600BF818885998508950B7FEB89EA93FE016C
:100D0600E95AFF4F0190F081E02DFA93EA93FE0134
:100D1600E95AFF4FFA93EA930E94E0005030089593
:100D26000E944305E0E3EA930C944805EA930E9487
:100D3600CB040C944305E991F991309639F08AEF8A
:100D460090E00197F1F7A8953197C9F708957B814F
:100D56006A81F981E88177FB770F67FD7160972FCC
:100D66009E5781F078F0983190F4AA27BB27882700
:100D760008948795B795A7959A95D1F7EA23FB230B
:100D8600682305C0E8947727EE27FF2766276F7745
:100D9600769508F4606877F9A991B9918991999146
:100DA600EA17FB076807790797FB0895D0DF09F470
:100DB6000895F6F79FEBAA27BB2780E862C10024B7
:100DC600AF0DB01D0895F195E195F0400895F095A9
:100DD60060957095E195FF4F6F4F7F4F0895EE0F29
:100DE600FF1FEE0FFF1F0895FE2FFF0FFF0B6F2F44
:100DF6007F2F08956F2F660F660B762F08950024B8
:100E060098E0AA0F001C0E1A10F40E0E01C0A16085
:100E16009A95B9F7EA2FA02D089551D0F0DF0EF478
:100E2600E19508950024112490E1AA0FBB1F001C30
:100E3600111C0E1A1F0A18F40E0E1F1E01C0A16007
:100E46009A9599F7FD01D001089545D0EBDF0EF490
:100E5600BADF08953F934F935F93002411244427EC
:100E6600552730E2AA0FBB1F881F991F001C111CB3
:100E7600441F551F0E1A1F0A460B570B28F40E0E59
:100E86001F1E461F571F01C0A1603A9559F7FD0165
:100E9600BC01D001CA015F914F913F910895E8943A
:100EA600A7FF02C0A1956894E7FDE195A8DFEA2FA8
:100EB6000EF4E1950895CEDFFD01BC010895E89496
:100EC600E7FF02C0E1956894A7FF04C0A19500F86A
:100ED600039400FA0895E894F7FF02C074DF68945B
:100EE600B7FF06C0A095B095119600F8039400FAD6
:100EF6000895ED91FC9111970895ED91FD916D91F5
:100F06007C91139708950590159065917491F00161
:100F160008957A936A93FA93EA930895182E862F82
:100F2600612D192E972F712D1B2EBF2FF12D1A2EE5
:100F3600AE2FE12D089530976040704009F070584B
:100F46000895552342F4503811F4E0FF04C0319659
:100F5600691F791F6BF050E8572711F45F93CDC0D6
:100F66005F3F31F0660F000C57956795752F089512
:100F76005F9300200AF0CDC0C6C050E8192E152296
:100F8600880F991F9527550F879550E8072E05223C
:100F9600660F771F7527550F67950895689401C0EA
:100FA600E8945F93F2DF703818F07F3F08F4A5C02D
:100FB60056E1571BAAF4519558300EF4593030F0CB
:100FC600EFEFFFEF6FEF7FE777F91AC0772755232B
:100FD600B9F0EE0FFF1F661F771F5A95D1F710C0A5
:100FE6007727583028F0EF2FF62F672F5850F9CF74
:100FF600552331F076956795F795E7955A95D1F78C
:1010060000200AF4E4DE5F910895689401C0E89434
:10101600309760407040B1F0002426F0772312F438
:101026000094D5DE172E7EE1112032F07A95EE0F70
:10103600FF1F661F111CF9CFEF2FF62F612D5F934F
:101046008ADF5F9108954F93AF01FD01DA01AB018D
:10105600BC01CA01402D012C142E4F910895EA0FB0
:10106600FB1F681F0895E095F0956095EF5FFF4FB1
:101076006F4F08955F9381DF903871F150E8152620
:1010860004C05F937ADF903839F1703821F1572F19
:10109600591B13F112F4D7DFFACF583118F0AA27EB
:1010A600BB278827583028F0AB2FB82F88275850F1
:1010B600F9CF552329F08695B795A7955A95D9F76F
:1010C600502D512562F0CBDF38F46795F795E795FB
:1010D600739513F41EC0B7DF3EDF5F910895EA1BD8
:1010E600FB0B680B51F010F40094BDDF6623A2F3EE
:1010F600EE0FFF1F661F7A95CBF7EE27FF276627B1
:1011060077275F910895EFEFFFEF6FE77FEF5F912E
:101116000895EFEFFFEF6FE77FE75F9108955F9325
:101126002CDF703851F3903841F301240894791F6D
:1011360023F41CF300203AF3ECCF0F921F932F9366
:101146003F934F93112722279927689FA0018F9FCE
:10115600302D410D591F6B9F300D411D591F8E9F1C
:1011660027D0BF9F25D06A9F23D0BE9F1DD0AF9F9B
:101176001BD0AE9F110D291F391F491F591FE32F81
:10118600F42F652F522F4F913F912F911F910F9062
:1011960066232AF0550FEE1FFF1F661F02C07395C8
:1011A6004BF2CFDE5F910895100D211D391F02C04D
:1011B600200D311D491F591F08955F93DEDE7038DB
:1011C60021F411200AF49FCFA4CF903809F495CFCB
:1011D60001240894970B1BF4D4F30020F3CF792F46
:1011E6001F932F933F934F931124112722273327C1
:1011F6004427552790E2AE17BF078607410730F010
:10120600AE1BBF0B860B410B089401C08894551F7B
:10121600221F331F111CAA1FBB1F881F441F9A952C
:1012260051F7F901612D4F913F912F911F9166233F
:1012360032F0550FEE1FFF1F661F7A9543F281DECF
:101246005F91089599239AF0772342F0971748F013
:1012560029F4AE17BF07860720F031F098948894DA
:101266000895989408940895189488940895772377
:10127600C2F7971798F3A9F7EA17FB07680788F3E9
:1012860099F3ECCF309760407040089510978040F6
:10129600904008955A934A933A932A931A930A933D
:1012A60008955D814C813B812A81198108810895C9
:00000001FF
